:020000040800F2
:1000000050050020D9000008C9170008F91600089B
:1000100000000000000000000000000000000000E0
:10002000000000000000000000000000131800089D
:10003000000000000000000011180008151800085A
:10004000EB000008EB000008EB000008EB000008E4
:10005000EB000008EB000008EB000008EB000008D4
:1000600000000000EB000008EB000008EB000008B7
:10007000EB000008EB00000800000000EB000008A7
:1000800000000000EB00000800000000000000007D
:10009000EB00000800000000EB000008EB00000887
:1000A000EB000008EB000008EB000008D51D00087D
:1000B000E51D0008EB000008000000000000000043
:1000C0000448854600F0F2FA004800474927000836
:1000D000C046C046500500200448804704480047F9
:1000E000FEE7FEE7FEE7FEE7FEE7FEE78D18000805
:1000F000C100000830B50B46014600202022012433
:1001000009E00D46D5409D4205D31D469540491B4B
:100110002546954040191546521E002DF1DC30BD94
:10012000F0B51FB40646002082B005464024019178
:1001300000901BE0019922460F46304600F09BF8E4
:10014000049A059B801A994110D3104619462246FD
:1001500000F081F8361A8F410197224601200021D4
:10016000009F00F078F838184D4100902046641E3A
:100170000028DFDC019B00982946324607B0F0BD1D
:10018000D2B201E00270401C491EFBD2704700222F
:10019000F6E710B513460A4604461946FFF7F0FF86
:1001A000204610BD70B502464A40D50F40004A00B7
:1001B000ED0740085208002814D0002A12D0C40DC0
:1001C000D30D41020120C0055202490A520AE41A25
:1001D000091812187D34914201D3641C00E04900D3
:1001E000002C01DA002070BD0023914201D3891A4E
:1001F0000343400849000028F7D100290AD0914262
:1002000002D10121C90705E0914201D2012101E09B
:100210000121C943E005C018401900F03DF870BD48
:1002200010B500229623114600F03EF810BDC20F13
:10023000D207400040080BD0C10D0723DB01C918CD
:1002400040020905400A1143C208400711437047A4
:1002500000200146704710B5202A04DB0146203AF1
:100260009140002010BD914020239C1A0346E3409A
:100270001943904010BD10B5202A04DB0846203AEF
:10028000D040002110BD0B46D340D0402024A21AFC
:1002900091400843194610BD002904DA401C49006A
:1002A00001D140084000704770B40024050C05D10E
:1002B0001024000402D1002921D01124050E01D1FF
:1002C00000020834050F01D10001241D850F01D162
:1002D0008000A41C002801DB4000641C002908D019
:1002E00020252E1B0D46F540A14000D001212943B9
:1002F000084301061B1B000ADB1D02D5002070BC51
:100300007047DB05181880180029F8DA401C4900EE
:10031000F5D170BC4008400070470000F0B50746BA
:100320000846584087B0C00F049048000E46590058
:1003300040084908BC1A884105D2384631461E4655
:1003400017460B4602465800400810434DD0300D6A
:10035000039040055900400D490D0590401A029048
:10036000402873DA18030121000B090508430190A6
:1003700004980092002806D01146019A49420020B4
:10038000904100910190029840210A1A0199009829
:10039000FFF761FF05460C466B4607CB00F098F966
:1003A000C0197141039A0E0D0023D71756401A4603
:1003B0007A40164344D0049A002A2DD0029A012A8A
:1003C000039A15DC1205C01A914101263605001C5E
:1003D0007141D20F059ED2070093019202962A46E0
:1003E000234600F095F907B0F0BD38463146FAE7EC
:1003F0001605234A0F46B218C01AB7410121090554
:10040000001C4F4100187F41114618187941E20F36
:1004100010436D19644113E0E2076D081543640849
:10042000C2071443039A01261205C01A91413605EA
:10043000001C7141CE07400830434908C0185141A3
:100440002A46234600F057F9CDE7FFE7049801223A
:100450004000C117121A00238B4104983146C4177B
:10046000381AA141EEE730B40124E407634030BC00
:1004700054E730B40124E407614030BC4EE700008B
:100480000000E0FFF0B51FB488B00B990998002474
:1004900048400999C00F490049080991C0070B99C4
:1004A0000090490049080B9109990898A64608430D
:1004B0001CD00B990A98084318D0099801244000D1
:1004C000420D4800410D099824050003000B20430C
:1004D00009900B980003000B20430B9050181C4907
:1004E0004018002201901446104605E00020014605
:1004F0000DB0F0BD032801DA034600E003239C465B
:10050000C11A0AAE0AE05F0008ADED5B4F00F75B71
:100510007D430027AA187C41491C5B1E6145F2DD22
:10052000410004AB5A522104120C0A43240C401C13
:100530000828DFDB01980290009970460191009035
:10054000059B049A0799069800F0E2F8D0E70000AE
:100550000DFCFFFFF0B50C465C4085B0E40FE407EE
:1005600003944C000026640859009446490802464A
:100570000296224321D062460A431ED06200570DE4
:100580004A000E032303550D012402462C4924057D
:10059000781B1B0B360B4018234326436146009003
:1005A0001C46501AB44103D30098401C009002E04E
:1005B000921800985B41002803DA0020014605B03C
:1005C000F0BD0020012109050746864611E064467A
:1005D0001D46141BB54106D36546521BB3417446F4
:1005E00007430C43A646CD07400849082843921804
:1005F0005B4105460D43EAD11046184313D06046CF
:10060000194650407140084306D06046101AB34165
:1006100006D20122002306E000220123DB0702E0CC
:100620000122D2435310009874460105381C6141E1
:10063000029C039D0019694100F05DF8BFE70000CE
:10064000FD0300004A0009030123090B1B051943A0
:100650000A4B10B5520D9A4202DA0020014610BD35
:10066000064B34339A4203DC9A1AFFF704FE10BD9E
:10067000034BD218FFF7EFFD10BD0000FF03000091
:10068000CDFBFFFF10B5002904DB0124E407404245
:100690008C412146002B04DB1C460123DB07524220
:1006A000A341994200D1904210BD0000064C0125A3
:1006B000064E05E0E36807CC2B430C3C984710340A
:1006C000B442F7D3FFF700FDA4270008C4270008B1
:1006D00010B5202A06DBCB170846203A1041C11777
:1006E0000B4306E00B461341D0402024A21A914050
:1006F0000843194610BD10B5002B08DA0024401C31
:10070000614192185B411A4301D14008400010BD7D
:10071000F0B51FB482B005460C0003D0084601F0C6
:1007200079FB02E001F076FB203002460090214682
:100730002846FFF790FD049B059A04460F46184390
:100740001143084314D0184610431BD00098402191
:100750000A1A18460599FFF78EFD05460E46009ABF
:1007600005990498FFF777FD084305D0012004E0C0
:100770002046394607B0F0BD0020C11705430E439F
:100780002C43374300990E986305401A7905E40A13
:1007900000220C43FD0A0A3002D500200146E9E799
:1007A0000105101969410C9C0D9D00196941FFF765
:1007B000A2FFDFE7704770B50024014620314A7977
:1007C000022A03D00421C163012418E002681368DF
:1007D0000E25AB431360026813685B085B0013606F
:1007E000436C1C221340012215469D40036C5D6042
:1007F0004A7100220A71816B002900D08847204687
:1008000070BD70B5044600F0C7F80546601C00D006
:10081000641C00F0C1F8401BA042FAD370BD000078
:10082000F8B500230124A2E027469F403A4070D04B
:100830004D68022D01D0122D14D1DD08AD002D1808
:1008400000952D6A5E07AC46F50E0F26AE46AE400B
:100850006546B543AC460E697546AE4065462E43C7
:10086000009D2E624D68012D05D0022D03D0112D63
:1008700001D0122D16D185680326AC465D00AE4628
:10088000AE406546B543AC46CE687546AE4065465B
:100890002E43866046680D79BE43ED06ED0F9D4000
:1008A0003543456006685F000325BD40AE46AE4354
:1008B0000D79B446AE07B60FBE4065462E430660BE
:1008C000C6687546AE438D68BD403543C5604D680A
:1008D000ED004BD5294D6E6B26436E639E08284D67
:1008E000B6007519AC46AD689E07360F0F27B740A6
:1008F000BD4305273F07B84201D1002715E0214F2E
:10090000B84201D1012710E01F4FB84202D102279F
:100910000BE02BE01D4FB84201D1032705E01C4F2F
:10092000B84201D1052700E00627B7402F436546AE
:10093000AF60184D2E684F689643FF0300D51643ED
:100940002E606E684F689643BF0300D516436E60F5
:10095000AE684F689643FF0200D51643AE60EE685E
:100960004F689643BF0200D51643EE605B1C0A68D1
:100970001546DD4000D057E7F8BD000000100240EA
:10098000000001400004005000080050000C00501E
:10099000001C00500004014001480068704700003E
:1009A0000800002002480168491C016070470000EF
:1009B0000800002010B508480024016840221143B7
:1009C0000160204600F00AF8002801D0012401E06F
:1009D00000F01CF8204610BD0020024070B505460E
:1009E00009487D210024C9000068FFF783FB00F05F
:1009F000F9FB002801D0012404E000222946501E02
:100A000000F01AF8204670BD0C0000200448416B2D
:100A1000012211434163816B0204114381637047DA
:100A200000100240C106C90E01208840014908603B
:100A30007047000000E100E010B500F0C7FE10BDF7
:100A4000F8B504460078544D800672D5524E002702
:100A5000403EB06BC00004D4B06BA9050843B0633E
:100A600001274E480168C90511D401688215114358
:100A70000160FFF791FF009005E0FFF78DFF0099FF
:100A8000401A642837D845480068C005F5D5326853
:100A90000321090560680A400140914208D08103A2
:100AA000890F032904D13168890301D50120F8BDDC
:100AB0002A69032109040A4022D0084090421FD02D
:100AC000207880061CD528692A6988430121C90439
:100AD0000A432A612A698A432A612861C0050FD521
:100AE000FFF75AFF009008E0FFF756FF0099411A00
:100AF0002B48814201D90320F8BD28698005F3D530
:100B000061688803800F032805D13268000582439D
:100B100001400A43326028690322616812041140CF
:100B200008432861002F04D0B16B012000078143E6
:100B3000B1632078C00705D0E868A168800880000C
:100B40000843E8602078800705D5E8680C218843D1
:100B5000E1680843E8602078400706D5E86803218B
:100B60008902884321690843E8602078000706D598
:100B7000E86803210903884361690843E860207835
:100B8000000606D5E868032189048843A169084363
:100B9000E8600020F8BD00004010024000700040F6
:100BA00088130000F8B50E4605007DD05348006854
:100BB000C007C00FB0420AD2504801684908490036
:100BC000314301600068C007C00FB04271D128787E
:100BD0004B4C800705D5E068F0218843A96808439D
:100BE000E0602878C00752D06868022817D0032830
:100BF00018D02168012818D08905002959DAE16840
:100C0000890889000143E160FFF7C6FE696807466D
:100C1000022912D003291CD0012926D033E02168F3
:100C20008903EAE721688901E7E74907E5E7FFF774
:100C3000B3FEC11B3348814223D8E0680007800F10
:100C40000228F4D123E0FFF7A7FEC11B2D48814203
:100C500017D8E0680007800F0328F4D117E0FFF7EA
:100C60009BFEC11B274881420BD8E0680007800F1C
:100C70000128F4D10BE0FFF78FFEC11B2148814210
:100C800001D90320F8BDE0680007800FF3D11B48AD
:100C90000168C907C90FB1420DD901684908490067
:100CA00031430160006800E003E0C007C00FB042BC
:100CB00001D00120F8BD2878400706D5E06807215B
:100CC00009028843E9680843E0602878000707D5EF
:100CD000E0680721C90288432969C9000843E06028
:100CE00000F036F8E168084A0906090F515CC8406F
:100CF000064908600020FFF771FEF8BD00200240A1
:100D00000010024088130000802700080C0000201B
:100D1000044805490068C968044A4905490F515CFF
:100D2000C84070470C0000200010024099270008BE
:100D3000044805490068C968044A8904490F515CA0
:100D4000C84070470C00002000100240992700089E
:100D500010B5184AD1680C20084004280BD0082888
:100D600010D00C2810D050680004410F0120C0039F
:100D7000491C884010BD1068C00601D50E4810BD42
:100D80000E4810BD0E4810BD88020E4B000F185CB7
:100D90000902D368890F491CDB0301D5084A05E025
:100DA0001268D20601D5044A00E0044A5043FFF716
:100DB000A1F910BD0010024000093D000024F4001C
:100DC00000127A0090270008FEB505007ED0FE4C88
:100DD000E7680C20E66807400120000406402878F8
:100DE000C00747D0082F05D00C2F0AD101200004DE
:100DF000864206D1206880033CD568680028E5D08B
:100E000038E0012069680004814203D12168014370
:100E1000216011E0052301221B04920499422168FC
:100E200002D111432160F1E7814321602168014033
:100E30000091206890432060686800280DD0FFF77B
:100E4000ABFD009005E0FFF7A7FD0099401A64286C
:100E50007AD820688003F6D50CE0FFF79DFD00905E
:100E600005E0FFF799FD0099401A6428F0D8206842
:100E70008003F6D42878800755D50923E868042F25
:100E80000DD00C2F01D1002E09D000283BD02168B5
:100E9000994301432160FFF77FFD064627E0216863
:100EA000490701D5002891D061681F2212029143A1
:100EB0002A6912021143616021689943014321604C
:100EC000FFF746FFE16809060A0F00E079E1BF4934
:100ED000895CC840BE4908600020FFF77FFD0028FC
:100EE00072D120E0FFF758FD801B0228B0D820689F
:100EF0004007F7D560681F21090288432969090264
:100F0000084360600FE02068400840002060FFF761
:100F100043FD064604E0FFF73FFD801B022897D8FB
:100F200020684007F7D42878C0065FD5002F0CD082
:100F3000A869002849D02068FF21013108432060BA
:100F4000FFF72AFD06462DE0C0E02068800502D5A7
:100F5000A8690028A7D06068072149038843296A47
:100F6000084360606068297F0002000A09060843A0
:100F70006060286A410B0120C003491C8840E16879
:100F800009060A0F9149895CC84091490860002010
:100F9000FFF724FD002817D128E0FFF7FDFC801B98
:100FA0000228A3D820688005F7D560680721490387
:100FB0008843296A084360606068297F0002000A4C
:100FC00009060843606011E0E1E02168FF2001307C
:100FD00081432160FFF7E0FC064604E0FFF7DCFCFC
:100FE000801B022872D820688005F7D42878794EB3
:100FF000000724D568690028306910D00121084312
:101000003061FFF7C9FC009005E0FFF7C5FC0099CF
:10101000401A02285AD830698007F6D50FE04008F8
:1010200040003061FFF7B8FC009005E0FFF7B4FC2A
:101030000099401A022849D830698007F6D42878E8
:10104000400765D500200290A06BC00006D4A06BBD
:10105000012109070843A063012002905E4801684E
:10106000C90511D40168821511430160FFF794FC92
:10107000009005E0FFF790FC0099401A642825D8FD
:1010800055480068C005F5D5FF20AA6801308242A6
:1010900003D131690143316111E001218902002A44
:1010A00007D005231B029A4203D132690A433261F9
:1010B000EFE7326982433261306988433061A86862
:1010C00000280FD0FFF768FC009007E05EE0FFF714
:1010D00063FC0099411A4148814257D83069800524
:1010E000F5D50DE0FFF758FC009006E0FFF754FC43
:1010F0000099411A3948814248D830698005F5D4B1
:101100000298002804D0A06B012109078843A0633E
:10111000686A002864D00C2F3ED0012636060228CB
:10112000206805D0B0432060FFF736FC05462FE06D
:10113000B0432060FFF730FC074604E0FFF72CFCCB
:10114000C01B022822D820688001F7D4E96AA86A67
:10115000E2680843296BFD231B049A4311430843AB
:10116000E060206830432060FFF716FC054604E08D
:10117000FFF712FC401B022808D820688001F7D531
:101180002EE0FFF709FC401B022801D90320FEBD19
:1011900020688001F5D423E00128F8D0E06801211F
:1011A0000904AA6A014091420BD10F218904EA6A1D
:1011B0000140914205D1032189050840296B8842ED
:1011C0000ED00120FEBD0000001002408027000864
:1011D0000C00002040100240007000408813000006
:1011E0000020EFE7094910B5401E884201D90120CF
:1011F00010BD074C60610321081F00F0E7FA0020D2
:10120000A06107202061002010BD0000FFFFFF004B
:1012100000E000E0F0B502462032137E012B15D02D
:10122000012717760223537605686C68AB68702631
:10123000B4430E68496826438024A34319436E6073
:1012400000688160577600201076F0BD0220F0BD66
:1012500070B5040005D025462035687E002802D0F0
:1012600006E0012070BD00202876204600F00AF834
:1012700002206876211D206800F032FB012068768C
:10128000002070BD00680449884204D10348816B86
:10129000102211438163704700100040001002408B
:1012A00070477047F8B502680446D06911689368C2
:1012B00005072D0F5BD0DD07ED0FFF2621360E4011
:1012C0002E4367D0C60706D0CE0504D50126166288
:1012D000E26F3243E267870702220426002F06DA14
:1012E000DF0704D027683A62E76F3743E7674707AD
:1012F00006D5DB0704D023681E62E36F1343E36760
:10130000020709D520220A402A4305D02368082273
:101310001A62E36F1343E367E26F002A2FD080065F
:1013200006D5880604D5216E002901D020468847BD
:10133000E06F21688968490601D4000724D520465A
:1013400000F09AFB20688168490619D5816840221F
:1013500091438160E06E002812D020498163E06EE5
:10136000FFF729FA00280AD0E06E816B06E08506B7
:1013700010D58D060ED5216E1CE020468847F8BD9D
:101380002046FFF78EFFF8BD2046FFF78AFF0020BA
:10139000E067F8BDC50208D55B0206D5012000054F
:1013A00010622046FFF77CFFF8BD030605D50B064B
:1013B00003D5616E0029E0D1F8BD4006FCD5480692
:1013C000FAD51368204640218B43136020216167C2
:1013D0000021616600F08FF9F8BD0000651A000871
:1013E00010B5040003D0606F002802D007E0012090
:1013F00010BD002170200155204600F027F8242060
:10140000606720680168490849000160204600F0D3
:101410009BFB0128ECD0606A002802D0204600F037
:101420008BFA206841680922D2029143416020680A
:1014300081682A229143816020680168012211435A
:101440000160204600F0DEFA10BD0000F0B587B064
:10145000044614216846FEF79AFE244F26680021B0
:1014600023480122022303240425BE421AD1466BDD
:1014700097033E434663C66A1643C662C06A02AE1D
:101480001040059060020090019332C60520694625
:101490000007FFF7C5F9002211461B20FFF7CCFA21
:1014A0001B201EE0134FBE421DD1866B01277F0417
:1014B0003E438663C66A1643C662C06A02AEC00770
:1014C000C00F05900C200090019332C6052069469C
:1014D0000007FFF7A5F9002211461C20FFF7ACFA20
:1014E0001C20FFF79FFA07B0F0BD00000038014054
:1014F0000010024000440040F0B5836F202B54D10F
:1015000000290AD0002A08D08568DC01A54206D14E
:101510000369002B03D1CB0701D00120F0BD0346A6
:1015200060331E7C012E40D001261E7441650146A9
:1015300040310A834A830022FF260266A54204D175
:101540000569002D13D11A4D0AE07F27002D09D01F
:1015500001263607B5420CD10569002D05D03F257F
:101560008D8307E00569002D01D08F8302E08E8313
:1015700000E08A83C2672221816701688D680126A5
:1015800035438D608168A14202D1016900290AD0EA
:10159000084901661A7400680168FF22213211436C
:1015A00001600020F0BD0449F3E70220F0BD000017
:1015B000FF010000F11A0008991A000810B5006830
:1015C000114988421ED111480178FF291AD141786A
:1015D00083784A1ED218C078D2B2904212D1080243
:1015E000C018FEF71DFE094948600949884209DD17
:1015F0000849FEF7D7FDFEF71AFE02460B4606A085
:1016000000F0F8FB10BD0000004400400000002086
:101610000000F0410000204164697374616E6365ED
:101620003A25332E31660A00FFB50446406F83B079
:1016300017460D4620285CD1002D0AD0002F08D077
:10164000A168C001814207D12069002804D1E807C0
:1016500002D0012007B0F0BD204660300290007C2F
:10166000012846D00298012101740020E067212062
:101670006067FFF791F926464036019037827782FE
:101680000120A1680003814202D12069002802D014
:101690002F46002511E000270FE000228021204680
:1016A00000F066FB002815D1002F15D0216838788E
:1016B00088627F1C708A401E7082708A019B00289D
:1016C00006980090E9D100224021204600F050FB0E
:1016D000002808D00320BDE728882168C005C00D78
:1016E0008862AD1CE6E7202060670299002008743C
:1016F000B0E70220AEE77047FEE7000008B50448F7
:10170000C16A01221143C162C06A1040009008BD45
:10171000001002401CB500240E4800940C490194AE
:10172000016007218460416001214461C160FFF7CD
:101730008FFD002801D0FFF73DF800946946054869
:101740000194FFF767FD002801D0FFF733F81CBDB7
:10175000001000401400002010B50C480A49016038
:10176000E1214902416000218160C1600161816124
:10177000C1610C22016242614162FFF731FE002823
:1017800001D0FFF717F810BD0038014050000020CD
:1017900010B50C480A4901604B21C9014160002184
:1017A0008160C16001618161C1610C22016242619D
:1017B0004162FFF715FE002801D0FEF7FBFF10BDC8
:1017C00000440040D0000020704700008307FF2243
:1017D000DB0E9A408907090E994000280BDA0007B2
:1017E000000F0838830808489B001818C369934302
:1017F0000B43C3617047830804489B001B1818689B
:10180000904308431860704700ED00E000E400E0FA
:101810007047704710B5FFF7C5F810BD30B599B0E7
:1018200034216846FEF7B3FC14210DA8FEF7AFFC87
:101830001C2112A8FEF7ABFC134801680322D20258
:101840009143C214891801600220009000241020E6
:1018500009940125049003956846FFF7B5FA0F2017
:101860000D9080200F900E951094002111940DA8DA
:10187000FFF798F9032012901494159412A8FFF71B
:10188000DFF819B030BD000000700040104801685A
:10189000821511430160C1680E4A1140C1600168A0
:1018A0000D4A114001608168490849008160016862
:1018B0000122920491430160C168FD221204914308
:1018C000C160002101610549C003886070470000C4
:1018D000001002400C40FF88F6FFF6FE00ED00E02D
:1018E00070B5026801239B07114C124D984203D03A
:1018F000A04201D0A84203D17026B2434E683243C1
:10190000984203D0A04201D0A84204D103231B0275
:101910009A43CB681A4380239A430B691A430260A7
:101920008A68C262096881620121416170BD00005C
:10193000000801400014014010B5818CC90707D090
:1019400001684A6801235B049A43836A1A434A6028
:10195000818C890707D501684A6801231B049A43D3
:10196000C36A1A434A60818C490707D501684A68EF
:1019700001239B049A43036B1A434A60818C090735
:1019800007D501684A680123DB039A43436B1A4376
:101990004A60818CC90607D50268916801231B0340
:1019A0009943836B19439160818C890607D501683F
:1019B0008A6801235B039A43C36B1A438A60818C54
:1019C000490612D503685A6801210905046C8A4347
:1019D00022435A60026C8A4207D10268516803238D
:1019E0005B059943436C19435160818C090607D507
:1019F00001684A680123DB04806C9A4302434A6011
:101A000010BD0000F8B500260446C667FEF7C4FF07
:101A1000054620680068124F000709D501212B46B2
:101A2000002249052046009700F0A2F900280DD1B8
:101A30002068006840070BD501212B46002289054C
:101A40002046009700F094F9002801D00320F8BD4B
:101A500020206067A067603426740020F8BD000075
:101A6000FFFFFF0110B5806A0022014640314A8322
:101A70004A82FFF716FC10BD01680A68FF23213374
:101A80009A430A6001688A68520852008A602021DD
:101A9000816700210166704710B5014640318B8B8C
:101AA000846F0268222C04D0906908210843906159
:101AB00010BD526A446D1A402280426D921C4265EC
:101AC0004A8B521E4A83498B0029F1D101680A686A
:101AD000FF2321339A430A6001688A685208520042
:101AE0008A602021816700210166FFF767FD10BD34
:101AF00010B5014640318B8B846F0268222C04D0D4
:101B0000906908210843906110BD526A1A40436DE4
:101B10001A70426D521C42654A8B521E4A83498B91
:101B20000029F1D101680A68FF2321339A430A6032
:101B300001688A68520852008A602021816700216A
:101B40000166FFF73BFD10BDF8B504462669A268A3
:101B5000E76932436669102000253E43236832431B
:101B600078491E68784F3E4016431E6023685A68C5
:101B700003263603B243E66832435A602368A269FB
:101B80008B4201D0266A32439E680B273F02BE4338
:101B900016439E606D4E23686D4AB3420CD1D268E5
:101BA0009207920F06D0012A38D0022A34D0032A95
:101BB00020D11EE001201DE0664EB3420AD1D2685A
:101BC0000C26324026D0042A28D0082A24D00C2AF9
:101BD00010D10EE08B420DD1D6680322920216403E
:101BE00018D001229202B61A18D0B61A14D0964212
:101BF00000D10820564A0126403A574FF6038B423F
:101C000036D100280CD002280DD0042812D0082884
:101C10001FD11CE00020EDE70220EBE70420E9E7FC
:101C2000FFF776F808E01068C00601D5384605E0F1
:101C30004A4803E0FFF78CF8002873D0626851002F
:101C40005118814205D81103814202D303E0304686
:101C5000F4E7012566E0010E060250080023301863
:101C60005941FEF75DFA03210902411A3C4A55E049
:101C7000E169B14232D1030000F0E3F809070A0D2F
:101C800006250606062B0600E3E7FFF741F81CE0F1
:101C9000FFF74EF819E010686168C00602D54808E1
:101CA000304A01E0304A48088018FEF723FA80B233
:101CB00001462E4A10399142CBD8511C01400007F1
:101CC000400F08432CE0FFF743F8616840004A08E2
:101CD000EAE76168012248081204E5E7030000F022
:101CE000B0F809070A0D06260606062C0600B0E71E
:101CF000FFF70EF81DE0FFF71BF81AE010686168A7
:101D0000C00602D54808C01902E014484A08101855
:101D1000FEF7F0F980B20146144A1039914298D882
:101D20002168C8600020206660662846F8BDFFF77D
:101D30000FF861684A088018EAE761684808801966
:101D4000E6E7000000480040F369FFEF003801407B
:101D5000401002400044004000093D000024F4000F
:101D6000FFFC0F0000127A000048E801EFFF0000BE
:101D7000FFB581B017460E4604460A9D09E0681C6F
:101D800007D0FEF709FE0499401AA8420CD8002D8E
:101D90000AD02068C1693046884318D00020B84274
:101DA000EDD0002005B0F0BD20680168FF22A1320F
:101DB00091430160206881684908490081602020C2
:101DC0006067A0670020603420740320EAE70120E8
:101DD000E5E7000010B50248FFF764FA10BD000007
:101DE0005000002010B50248FFF75CFA10BD00005B
:101DF000D00000200FB410B503A9044B044A029888
:101E000000F0F6F810BC08BC04B018472D270008F5
:101E1000100000202021020C01D010211046020ADF
:101E200001D010460839020901D01046091F820866
:101E300001D01046891E420801D0881E7047081A3A
:101E4000704730B47446641E2578641CAB4200D2DF
:101E50001D46635D5B00E31830BC184702E008C80C
:101E6000121F08C1002AFAD170477047002001E014
:101E700001C1121F002AFBD170470000F0B51FB44A
:101E800086B00998089A030D0021024314D05148E6
:101E9000514A1818504305141198012810981AD067
:101EA000281A401C00264D4F4D4900960191049080
:101EB000002812DA444211E01198012449A30128B4
:101EC00001D11098C1430698119A84600360C260E2
:101ED00041600BB0F0BD4042E4E70446210500201C
:101EE0003F4A001C51410391029012E0E00707D0E5
:101EF00032463B4601990098FEF7C4FA01910090E2
:101F000032463B4610461946FEF7BCFA06460F46D7
:101F10006410002CEAD10498039B0028029A0999C6
:101F2000089806DAFEF7AEFA019B009AFEF7AAFAC5
:101F300005E0FEF70FFB019B009AFEF70BFB044642
:101F40000E460022284BFEF79DFB03D80020C0431D
:101F5000014607E00022254B20463146FEF7DEF918
:101F6000FEF770FB102409E0002C0ADB0A22002394
:101F7000FEF7D6F8079B30321A55641E02460A4314
:101F8000F2D11122641C079B121B1C19119B012BFF
:101F900003D0012308430ED10AE0084304D01120E6
:101FA00010900020119077E71098151A6D1E0BE025
:101FB0001098824202DD00236D1C03E0824201DAA8
:101FC00000236D1E002BEED0069811998260C1602F
:101FD00030C07EE701FCFFFF104D00000000144000
:101FE0000000F03F300000000000F0430000E03F40
:101FF000FFB597B0064600251BE2252876D10024C0
:102000002746F749049400E00443761C3278012007
:10201000203A90400842F7D130782A280ED0022288
:10202000307801463039092916D804990A235943D2
:10203000303940181443761C0490F1E7189802C810
:1020400004911890002904DA012040030443484217
:10205000049002200443761C30782E2814D10420EA
:1020600004437078761C2A2809D11898761C80C8F9
:10207000189009E00A214F43303FC719761C307889
:10208000014630390929F5D930786C2810D006DCA2
:102090004C281AD068280ED06A2817D104E074287A
:1020A00013D07A2812D110E00120400504430CE03F
:1020B0000121090501E0032109050C4371788142E2
:1020C00003D1012000052418761C761C3078662880
:1020D0000BD013DC58287DD009DC00287BD04528A4
:1020E000F6D04628F4D047281AD1A9E118E0632891
:1020F00035D0642870D0652812D1A1E170286CD049
:1021000008DC6728F1D069287DD06E280DD06F28B3
:1021100006D1BCE073282ED0752873D0782859D00A
:102120001A9A199990476D1C82E16002400F0228AB
:1021300009D003280DD00428189801680DD00D602F
:10214000001D189074E11898EA1701680D604A6044
:10215000F6E7189801680D80F2E70D70F0E718981F
:102160006A4601781172001D18900020507202A872
:102170000090012005E0189802C8189000200091F6
:10218000C04361070ED5002101E00199491C01916E
:10219000B94213DA8142F8DB019A0099895C00297F
:1021A000F3D10BE0002101E00199491C019181422A
:1021B000FADB019A0099895C0029F5D1019904980C
:1021C0001A9B471A21463846199A00F099FA401985
:1021D000019903E051E030E115E050E0451807E0D7
:1021E000009800990078491C00911A9A1999904713
:1021F0000198401E0190401CF2D1214638461A9B9E
:10220000199A12E137E00A20002100900191600242
:10221000410F022907D0189A01CA1892C217944692
:10222000032908D00AE01898C01DC108C90005C9D3
:102230001891944607E000B2C2179446042902D1CF
:1022400040B2C1178C4600226146944506DA0A4620
:102250000021404291418C462D2102E0210504D508
:102260002B216A461173012103E0E10701D02021EF
:10227000F7E7029156E00A200AE0102008E010205B
:1022800000900021042004430191082703E0082066
:102290000021019100906002410F022907D0189A95
:1022A00001CA189200229446032908D008E0189821
:1022B000C01DC108C90005C91891944603E080B249
:1022C000042900D1C0B20021029121072AD531781A
:1022D0000D91702906D0009A1021019B4A401A43A3
:1022E00005D00EE040216A461173012108E06146E5
:1022F000014306D030216A4611730D9951730221B2
:102300000291009A0821019B4A401A430AD1614672
:10231000014301D1610705D530216A4611730121BE
:102320007F1E02913178582904D02EA10E910DA95B
:102330000D910DE030A1F9E76146019B009AFDF790
:10234000EFFE0E9B8C469B5C0D9A521E0D921370F5
:1023500061460143F0D10D9805A9081A203001907B
:10236000600703D501200004844300E001270198A1
:10237000874201DD381A00E00020019900904118E1
:10238000029809180498401A0490E00306D42146E4
:102390001A9B199A049800F0B3F94519002706E032
:1023A00003A81A9AC05D199990476D1C7F1C02986A
:1023B0008742F5DBE0030CD521461A9B199A049855
:1023C00000F09EF9451904E01A9A302019999047B7
:1023D0006D1C0099481E00900029F5DC1FE00000EC
:1023E00009280100303132333435363738396162EB
:1023F00063646566000000003031323334353637AF
:102400003839414243444546000000000D980D997B
:102410000078491C0D911A9A199990476D1C0199E1
:10242000481E01900029F1DC4DE100F059F94519F1
:10243000761C3078002800D0DFE528461BB0F0BDC0
:10244000600700D406271898C01DC108C900486855
:102450000A680831C30FDB071891190001D09CA14D
:1024600008E0210501D59BA104E0E10701D09AA174
:1024700000E09AA14300109130785B0865280CD0E9
:1024800006DC452809D046281DD0472841D141E027
:10249000662818D067283CD13CE00021112F01DBD1
:1024A000112000E0781C0191009008A911A8FFF705
:1024B000E5FC139905910021119A15927F1C129841
:1024C0000197009150E00120C00703900120019086
:1024D00008A9009711A8FFF7D1FC139A1499059247
:1024E0000022119B009212981593059A01920029DF
:1024F00001D0104602E0791C40180190381A01D52D
:10250000019804E04042401E0090781C0190C01BDE
:10251000029043E0012F00DA01270021112F01DD95
:10252000112000E038460191009008A911A8FFF79A
:10253000A5FC13990591119A00211298159200910A
:10254000019721070CD40599B94201DB019900E0FC
:102550000191012904DD159A491E515C302906D0EC
:10256000B84201DA011D05DA0121029115E0019955
:10257000491EEDE7002805DC0099411800910199FA
:10258000091A03E0019A411C914200DD0191009972
:10259000401A401C02900120C0070390200706D477
:1025A00002990198814202DB0020C0430290002082
:1025B0006946C87707AF012103980337C9078842E6
:1025C00024D0022011902B201290039800280CDABE
:1025D000404203902D20129007E00A210398FDF756
:1025E00089FD30317F1E039039701199481E11907A
:1025F0000029F2DC03980028EFD1791E12980870A8
:102600003078202108404530BF1E387006A8C01B16
:10261000C01D039010980078002800D00120019977
:1026200041180298C0170918039809180498401A0D
:10263000401E0490E00306D421461A9B199A049880
:1026400000F05EF8451910980078002803D01A9A17
:10265000199990476D1CE00324D521461A9B199ABD
:10266000049800F04DF845191CE00098002807DB9D
:1026700000990598884203DD1598405C199901E09E
:10268000199930201A9A904700986D1C401C0090B0
:102690000298401E0290002804D11A9A2E201999FF
:1026A00090476D1C0199481E01900029DDDC05E072
:1026B00038781A9A7F1C199990476D1C0399481E07
:1026C00003900029F4DC21461A9B199A0498ACE681
:1026D0002D0000002B000000200000000000000082
:1026E000F8B5044600251E461746880404D405E0C4
:1026F00039462020B0476D1C641EF9D52846F8BD28
:10270000FFB50446002581B01E46C80301D5302719
:1027100000E02027880404D505E038460399B04737
:102720006D1C641EF9D5284605B0F0BD01B5044BFB
:10273000012269460348FEF777FF009808BD0000B4
:10274000FFFF000050000020FEF734F9FFF766F8A5
:10275000FEF7D4FFFFF700F8FEF7DCFFFFF718F8ED
:10276000044C042204490548FEF7C6FE2046FEF745
:1027700048F8F6E79411000000000020D000002087
:102780000000000000000000010203040607080921
:10279000030406080C10182030000000000102039A
:1027A00004000000C42700080000002014000000FE
:1027B0005C1E0008D8270008140000203C0500001B
:1027C0006C1E000800000000000000000000000077
:0827D0000000200000000000E1
:04000005080000C12E
:00000001FF
